:020000020000FC
:1000000000C001E107BB06E108BB0FED0DBF01E039
:10001000902E88249AD0112772D0C02EA8D1B199E1
:10002000FECFA8ECBB27DED0119729F0B19BFBCF08
:10003000C4988BD035C0C498ACEDB5E0D3D011973F
:1000400019F0B19BFBCFB2C1C49AB19BFECF7DD05A
:100050000AE05CD0B199FECFA4EFBB27C3D01197C3
:10006000A9F0B19BFBCF71D0C39481D10C2D00308E
:1000700011F410E009C0013011F415E005C00230A0
:1000800011F412E001C011E040D0E4CF0AE23ED00A
:10009000C49AB19BFECF59D00C2D112729D0BFCFC8
:1000A000A6D0C49A062D0295302F307F062D252D1F
:1000B00022950295207F0F70202B052D142D12956F
:1000C0000295107F0F70102B042D02950F7066D0D3
:1000D000122D103041F012951F70103009F015D01C
:1000E000122D1F7012D0132D12951F700ED097CFA6
:1000F000E199FECF0DBB1EBBE29AE19A0895E1990A
:10010000FECF1EBBE09A0DB3089529D000FF09D0A1
:1001100000FD09D01AD006950130C1F716D015D0D0
:10012000089542E001C046E030E3542F662726E000
:1001300050FFC09850FDC09A6A95F1F72A95E1F7F3
:100140005A95A1F73A9589F7089530E366272CE090
:100150006A95F1F72A95E1F73A95C1F708951030BD
:1001600009F40FE3113009F40EE3123009F40CE343
:10017000133009F408E3143009F400E3153009F4EE
:1001800000E2163009F401E2173009F403E21830F6
:1001900009F407E2193009F40FE2089540E200245F
:1001A0001124222433244424330F221F111F001F43
:1001B00010F4316001C03E7F441C331C221C111C12
:1001C000001C4A9509F40DC0EFEFE39550815D5F87
:1001D00053FD50835081505D57FD5083E430A9F7A3
:1001E000E3CF0895E0E0FAE03197F1F7089507E0F2
:1001F00003BF07E3002E03E0102E06E0202E662446
:100200005524442482BE00000000000000000000CD
:10021000000009181808280859F0762C62B66714EF
:1002200020F0000000000000F4CF590C481CF1CF72
:10023000089507E003BF04E3002E00E6102E00E05F
:10024000202E66245524442482BE09181808280844
:1002500079F3762C62B6671420F0000000000000ED
:10026000F4CF590C481CF1CF08950027072906291F
:100270000529042908950027072B062B052B042B9D
:100280000895F9DF11F1F1DFF9F03324222411246C
:100290000024770C661C551C441C00E2331C221CF5
:1002A000111C001C371626061506040630F0371AF6
:1002B000260A150A040A089401C08894771C661C53
:1002C000551C441C0A9551F708950895CEDF19F185
:1002D000D2DF29F477246624552444240895332456
:1002E00022241124002400E2330C221C111C001CC7
:1002F000771C661C551C441C40F4370E261E151E28
:10030000041E781C681C581C481C0A9569F7732C3D
:10031000622C512C402C0895770E661E551E441EEB
:100320000895771A660A550A440A089577166606EC
:10033000550644060895072D772E702F062D662E3C
:10034000602F052D552E502F042D442E402F08953B
:10035000442755276A2D7B2D94DFB8DF409260003B
:1003600050926100609262007092630008950C2DBB
:10037000043010F000E0C02E003029F407E2A02E77
:1003800000E1B02E0895013029F403E1A02E08E821
:10039000B02E0895023029F407E0A02E00EDB02E13
:1003A000089503E0A02E08EEB02E089542DF7724D2
:1003B000CFDF3FDF77244092640050926500609267
:1003C00066007092670040916000509161006091FA
:1003D000620070916300AADFA0F4ADDFA2DF40E00D
:1003E00050E061E070E0A2DF00F1F9F040906400BD
:1003F000509065006090660070906700A9DF91DE04
:1004000014C08FDF40E050E06A2D7B2D8FDF08F4B1
:100410000CC0409064005090650060906600709041
:10042000670096DF7EDE91DE7CDEB199C2CFC49A92
:0A0430008CDEB19BFECF89DEF2CD19
:00000001FF
